:10000000F528A0008417800484138E010C1C8E0038
:1000100010200319F02810200319F0281020F028D0
:1000200020088E0601308C008D01000820050E0688
:10003000031D08008C0A03198D0F15280800910173
:1000400090009F1727308F001030322003308F0030
:10005000E83032208F01643032208F010A303220A4
:1000600010083D288E0011088D0010088C00D42047
:100070000C08031D9F139F1B0800303E92002208AE
:1000800084000930930003104A20920C930B4428FB
:1000900003144A2884139F1D5928000820041F1D9B
:1000A00020068000841700082004031C200680001E
:1000B000642800082004031C20061F192006800065
:1000C00084172009800564281F0D06398C006D20D7
:1000D0008D008C0A6D200000C02800308A000C08BA
:1000E0008207013475340334153400343C340C3445
:1000F000D9348F00220884002009A02084138F089F
:100100000319F028F03091000E0880389000F0308C
:1001100091030319910003198F030319F028902804
:10012000A32003010C1820088E1F20088E08031935
:100130000301900F9D28800684289E2800008728B0
:1001400084178005F0280D080C0403198C0A8030F0
:100150000C1A8D060C198D068C188D060D0D8C0D44
:100160008D0DF0288F018E00FF308E07031C8F0746
:10017000031CF02803308D00DF30C020B4288D012F
:10018000E83E8C008D09FC30031CC9288C0703183D
:10019000C6288C0764008D0FC6280C18CF288C1C2D
:1001A000D3280000D328080091019001103092005C
:1001B0000D0D900D910D0E0890020F08031C0F0FEE
:1001C00091020318EA280E0890070F0803180F0F72
:1001D000910703108C0D8D0D920BD8280C08F02878
:1001E0008313031383126400080083160330850011
:1001F00008308600831206108316061083128610BC
:100200008316861005308312A2000830A000043047
:100210009F00FE303E2001303E2003308F00E8304A
:10022000B3200530A2000830A00004309F00FE304B
:100230003E2080303E2052303E2061303E206430EF
:100240003E2069303E206F303E2020303E2043303B
:100250003E206F303E206E303E2074303E207230A3
:100260003E206F303E206C303E200630A200103021
:10027000A00064308E000A30792032308E000530C4
:10028000792046308E000A30792032308E000230DC
:10029000792003308F00E830B3200530A200083009
:1002A000A00004309F00FE303E2080303E206330AE
:1002B0003E2068303E2061303E206E303E206E3061
:1002C0003E2065303E206C303E202D303E203130C7
:1002D0003E203A303E2020303E2020303E2020304C
:1002E0003E2020303E2020303E2020303E20053071
:1002F000A2000830A00004309F00FE303E20C03035
:100300003E2043303E2068303E2061303E206E303B
:100310003E206E303E2065303E206C303E202D3039
:100320003E2032303E203A303E2020303E202030E9
:100330003E2020303E2020303E2020303E20203005
:100340003E2001308C0005308400013001200C0873
:10035000A40001308C0005308400023001200C081C
:10036000A5000530A2000830A00004309F00FE3038
:100370003E208A303E2024081F2020303E2020309E
:100380003E2020303E200530A2000830A00004307E
:100390009F00FE303E20CA303E2025081F2020301E
:0C03A0003E2020303E2020303E20A129CD
:02400E00F53F7C
:00000001FF
